:100000004528A00014200C080D04031940283A20AC
:1000100084132008800664000D280E288C0A03191A
:100020008D0F0B2880064028FF3A84178005402852
:100030008F018E00FF308E07031C8F07031C4028A2
:1000400003308D00DF3026201A288D01E83E8C0019
:100050008D09FC30031C2F288C0703182C288C07D3
:1000600064008D0F2C280C1835288C1C39280000B2
:10007000392808008C098D098C0A03198D0A08009B
:100080008313031383126400080086130613861279
:100090000D30A4008C30A6008C30A5008C30A70059
:1000A00052204A280130A80064000B3028020318AF
:1000B000722826088C008D010630840080300120D3
:1000C00025088C008D01063084004030012027086F
:1000D0008C008D0106308400203001202408182077
:0600E000A80F54280800DF
:02400E00F53F7C
:00000001FF
